:020000040000FA
:020000000528D1
:08000800F7298312850107307E
:1000100099008316FF2390003F309F001F3085001A
:10002000203095008312A401AD019C21A41C1A2844
:100030002808B12128080A3C0319152828080D3C76
:1000400003192D282D08043C031915282E302D07DF
:10005000840028088000AD0A1528A41C31280A3025
:10006000B1212D08043C031D1428B301AD012E302D
:100070002D07840033083307330733072D0750203B
:1000800080120002031D4A28AD0A2D08043C031DFE
:1000900037287528B30A3308093C031D362814286D
:1000A0008207543445344D34503456344534523438
:1000B00053345334543441345434533457344F3418
:1000C0004E34533457344F3446344434493447342F
:1000D000493441344E3441344C344534433448344B
:1000E0004F345434523455344E34B30803199128E4
:1000F000B30303199328B3030319A428B303031903
:10010000D228B3030319D428B3030319D628B303A1
:100110000319DC28B3030319E228B3030319E72802
:100120001428F82014289630EC2014285034693410
:1001300074346834203456346534723431342E3497
:1001400031340D340A34003483169F19AF288312DA
:10015000BC30EC20C530051ECB30EC2014288312B7
:10016000B330EC20142841346E3461346C346F3475
:1001700067340D340A3400344434693467346934E4
:10018000743461346C34283400344F344E342934A0
:100190000D340A3400344F344634463429340D3497
:1001A0000A340034051614280512142883169F11EA
:1001B000051283122414142883169F150516831222
:1001C000241014282408A401A414A4061428F82038
:1001D000E821851DE7281428AB00AC012B082C076B
:1001E000F720003E03190800B121AC0AEE28820076
:1001F000813027213E08B5004008B4008530272112
:100200003E08B7004008B600893027213E08B900F3
:100210004008B800241812298D3027213E08BB0061
:100220004008BA0000307A212C30B12101307A2107
:100230002C30B12102307A21241822292C30B1210E
:1002400003307A210D30B1210A30B1210800C100FC
:10025000BE01BF014030C20041089F00D2219F145F
:100260009F1830291F1083161E08BD0083121E0818
:10027000BC003D08BF070318BE0A3C08BE07C20BFE
:100280002C29C001BE1F4E29C009BD01BC013F0879
:10029000BD02031CBC033E08BC0252293F08BD003E
:1002A0003E08BC003D08BF003C08BE000310BE0C69
:1002B000BF0C682168216821682168214030BF0790
:1002C0000318BE0ABF0DBE0D0310BE0CC00D080002
:1002D0000310BE0CBF0C3D08BF070318BE0A3C0844
:1002E000BE070800A5018002031C7829A50A73290E
:1002F000800708008400840734308407801F822927
:100300002D30B121840A64307221250803198A290D
:10031000303EB1210A307221250803199129303E5F
:10032000B1210008303EB1212E30B121840330309C
:1003300000183530B1210800A80185199D29851DB7
:100340009F29CB210830A60000000000000000001B
:100350000000C3210310851D0314A80CA60BA929B6
:100360000800A9000830A7008516CA21A90C031CA3
:10037000851603188512C421A70BB6298512CA2138
:10038000080085120800000000001E30AA00AA0B19
:10039000C7290800CB210D30AA0000000000AA0BDD
:1003A000CF2908000530A300A30BD4290800203072
:1003B000A00000000000A00BDB2908001F30A100F6
:1003C000A10BE0296130A100D721A10BE42908008D
:1003D0006330A200DE21A20BEA295E30A200D72101
:1003E000A20BEF290630A200A20BF4290800090095
:02400E00C43FAD
:00000001FF
